:020000040000FA
:10000000802C0020F902000001030000030300001F
:1000100005030000070300000903000000000000C2
:100020000000000000000000000000000B030000C2
:100030000D030000000000000F030000110300008A
:100040001303000079060000390A000013030000C2
:100050001303000013030000F50300001303000066
:10006000D509000013030000130300001303000070
:100070001303000013030000130300001303000028
:10008000130300000907000013030000130300001E
:100090002D070000310700001303000013030000C8
:1000A00013030000130300001303000013030000F8
:1000B0001303000013030000000000000000000014
:1000C00013030000130300001303000013030000D8
:1000D00013030000130300001303000013030000C8
:1000E00013030000130300001303000000000000CE
:1000F00000000000130300000000000013030000D4
:1001000000000000000000000000000000000000EF
:1001100000000000000000000000000000000000DF
:1001200000000000000000000000000000000000CF
:1001300000000000000000000000000000000000BF
:1001400000000000000000000000000000000000AF
:10015000000000000000000000000000000000009F
:10016000000000000000000000000000000000008F
:10017000000000000000000000000000000000007F
:10018000000000000000000000000000000000006F
:10019000000000000000000000000000000000005F
:1001A000000000000000000000000000000000004F
:1001B000000000000000000000000000000000003F
:1001C000000000000000000000000000000000002F
:1001D000000000000000000000000000000000001F
:1001E000000000000000000000000000000000000F
:1001F00000000000000000000000000000000000FF
:10020000DFF80CD000F0C6F8004800474D2A000087
:10021000802C002030B4044654E8000F0D4644E81A
:100220000053002BF8D1156030BC704730B4044641
:1002300054E8000F40EA010544E80053002BF7D1D1
:10024000156030BC704730B4044654E8000F00EA33
:10025000010544E80053002BF7D1156030BC70470E
:1002600030B4044654E8000F80EA010544E8005326
:10027000002BF7D1156030BC704730B4044654E809
:10028000000F00EB010544E80053002BF7D1156087
:1002900030BC704730B4044654E8000FA0EB0105B1
:1002A00044E80053002BF7D1156030BC704770B4A0
:1002B00004464FF0000054E8006F0D68AE4207BFDF
:1002C00044E80023012044E800630E60002B1CBFBB
:1002D0000020F0E770BC704730B4044654E8000FCB
:1002E00088422CBF451A054644E80053002BF5D13F
:1002F000156030BC7047000006488047064800473C
:10030000FEE7FEE7FEE7FEE7FEE7FEE7FEE7FEE7C5
:10031000FEE7FEE7A5070000010200000048704765
:100320001C74000040EA01039B0703D009E008C9E0
:10033000121F08C0042AFAD203E011F8013B00F8AA
:10034000013B521EF9D27047D2B201E000F8012BF6
:10035000491EFBD270470022F6E710B513460A4645
:1003600004461946FFF7F0FF204610BD421C10F866
:10037000011B0029FBD1801A704730B504460020CC
:10038000034600E05B1C934203D2E05CCD5C401B63
:10039000F8D030BD064C074D06E0E06840F00103A0
:1003A00094E8070098471034AC42F6D3FFF72CFFCF
:1003B000BC740000DC74000030B58C1810F8012B00
:1003C00012F00F0301D110F8013B120906D110F809
:1003D000012B03E010F8015B01F8015B5B1EF9D112
:1003E00001E001F8013B521EFBD1A142E6D30020FF
:1003F00030BD00002DE9F04F00268DB0DFF8A08160
:10040000B14604964FF48075012437460596284678
:1004100003F0CAFA38B1D8F80403204203D02846C2
:1004200003F0B8FA26432D1D64007F1CADB2082FDF
:10043000EDD34FF4BE74204603F0B6FA48B120461F
:1004400003F0A8FA46F0004604AA0221002003F0B7
:100450008BFA544C16F0FF0F15D0012700253742B8
:100460000DD008EB8501D1F81005D1F81015C0F3B7
:10047000052054F82520C1F3014102B190477F00C7
:100480006D1C082DEBD3002E7EDA0020CDF82890CD
:10049000411E0DF1100B07AACDF82C9042F8201048
:1004A000401C91460228F9D300252E46A11911F8C7
:1004B000607F91F9000027F0C008401C40D007A9D8
:1004C000404602F025FD40B34FEA971A404600F03F
:1004D00059FC54F820701FB1BAF1030F03D006E0A5
:1004E000BAF1030F2CD10AA9404602F019FD02A867
:1004F000CDF8088003F0E6F9029900EB8100D0F80E
:10050000000704A9C0F301400290404602F000FD3C
:100510000028029802D0022802D011E003280FD14F
:10052000BAF1030F08D10298022833D002214046C5
:1005300003F0A1F96D1CEDB217B151464046B84722
:10054000761C042EB2D3002D21D001AA0221002056
:1005500003F00AFA00205A460DF1040152F8206017
:1005600051F82030B34217D000200AAE4FEA0903F9
:1005700051F8207042F8207056F8207043F820702F
:10058000401C0228F4D300E001E0002D8CD10DB016
:10059000BDE8F08F0321CAE7401C0228DED3F6E74E
:1005A000006000408C01002000F01F0201219140FA
:1005B0004009800000F1E020C0F88012704700F090
:1005C0001F02012191404009800000F1E020C0F8A5
:1005D0008012704700F01F02012191404009800005
:1005E00000F1E020C0F88012704700F01F020121E6
:1005F00091404009800000F1E020C0F8801270476F
:1006000000F01F02012191404009800000F1E0202C
:10061000C0F88011704700F01F020121914040098D
:10062000800000F1E020C0F80011704700F01F02C8
:10063000012191404009800000F1E020C0F8001144
:10064000704700F01F02012191404009800000F135
:10065000E020C0F8001270474907090E002806DAAA
:1006600000F00F0000F1E02080F8141D704700F149
:10067000E02080F80014704770B5204D28696C7830
:10068000401C2861687D10B11D4800F0B7FC287837
:1006900003281AD11B48D0F80C01B0B1012C04D0AA
:1006A000022C0AD01648123023E02869032816D0FD
:1006B0001348083000F0A2FC11E02869022812D08B
:1006C0000F480D3000F09AFC0DE0032C0FD2012CE6
:1006D00005D0022C07D0BDE8704004F023BCBDE873
:1006E000704004F04BBCBDE8704004F05DBE0448AF
:1006F0002830BDE8704000F081BC000030090020C7
:1007000038030A000010004007480021C0F84011DB
:10071000C0F84411C0F84811C0F84C11C0F80011DD
:10072000C0F8041106F0C0BB0010014006F02EBB5B
:1007300030B51B4C85B00025012080F31088D4F81B
:10074000D40038B3D4F8D00000EB800004EB800074
:1007500001798DF800108168C26803694069CDE9AC
:100760000330CDE90112D4F8D400401EC4F8D400FF
:10077000D4F8D000401CC4F8D000D4F8D0000A2827
:1007800001D3C4F8D050002080F310882168684657
:100790008847D1E7002080F3108805B030BD000005
:1007A0004C09002030B54FF0805000228300D0F873
:1007B0003011C3F80C21C3F81021624B1A60624B50
:1007C0001B68624C2360604B1B1D1B68241D23604B
:1007D0005D4B08331B68241D23605B4B0C331B6887
:1007E000241D2360584B10331B68241D2360564B77
:1007F00014331B68241D2360534B18331B68534C60
:1008000020342360504B1C331B68241D23604E4B47
:1008100020331B68241D23604B4B24331B68241D8D
:100820002360494B28331B68241D2360464B2C331F
:100830001B68241D2360444B30331B68434C4034F9
:100840002360414B34331B68241D23603E4B3833F7
:100850001B68241D23603C4B3C331B68241D236014
:10086000394B40331B68241D23600124082902D121
:10087000D0F8343113B1082904D006E0354B34499F
:10088000196005E0D0F8343113B1082904D006E02E
:10089000314BFB21196005E0D0F8343113B1082940
:1008A00008D00EE090F858322C48016863F3030139
:1008B000016002E0D0F834311BB929494FF40070CF
:1008C000086028480168C90702D06FF00101016083
:1008D0002548016841F470010160BFF34F8FBFF3F9
:1008E0006F8F4FF01021D1F80002002803DBD1F800
:1008F0000402002822DA1D4B1C601D480468002CED
:10090000FCD01224C1F800420568002DFCD0C1F8CB
:10091000044201680029FCD01A6001680029FCD05B
:10092000BFF34F8F10487C380168124A01F4E06130
:1009300011430160BFF34F8F00BFFDE70F490E4821
:10094000086030BD380500400404001020C5004098
:10095000488103008C56004018F50040E40E00402A
:10096000409602400004004088ED00E004E50140AC
:1009700000E401400400FA050090D003D0000020FC
:10098000124A10B50021104B126809E053F82140BB
:10099000844203D10E4800F031FB13E0491CC9B278
:1009A0009142F3D3084A002112F1180201EB01131E
:1009B00002EB4303834201D1012010BD491CC9B29F
:1009C0000629F3D3002010BD980B00204001002021
:1009D000EC00030070B5144E4FF48030C6F80803E5
:1009E0000025C6F84051114C606810B9104800F05D
:1009F00005FBA57062680123656073640D4801689A
:100A0000001F00681430B1F5804F04D2B0F5404F9C
:100A100001D9637005E0814201D3012000E000208C
:100A20006070BDE870401047008000401801002051
:100A3000E5000400448500400148006800470000CC
:100A40002000002002E008C8121F08C1002AFAD1C5
:100A500070477047002001E001C1121F002AFBD13E
:100A60007047000072B605F027FA00BF05F07AF86B
:100A70000028FBD1104C0121208801EB00400FA180
:100A800005F07CF910480068C00700D000BE20883F
:100A9000022101EB00400DA105F070F9BFF34F8F6B
:100AA0000948E43801680D4A01F4E061114301602E
:100AB000BFF34F8F00BFFDE758010020466174610E
:100AC0006C206572726F7200F0ED00E05379737400
:100AD000656D207265736574000000000400FA05FE
:100AE0000EB500210091CDE901106A4644F20100E3
:100AF000FFF7B8FF0EBD00F003B800F009B8000022
:100B000072B602480168491C016070473C00002031
:100B100003490868401E086000D162B670470000B3
:100B20003C00002070B5054608680C46411C04D006
:100B300002F0F2FE206802F08AFE6068411C02D0DA
:100B4000002102F072FE2968A069C1F82405607DC9
:100B5000227D29681043C1F86C05D4E90012286889
:100B6000C0F81425C0F80C15207D012814D1A06808
:100B7000411C02D0002102F058FEE068411C04D064
:100B800002F0CAFEE06802F062FED4E902122868B0
:100B9000C0F80825C0F8101570BD70B50546086886
:100BA0000C46411C04D002F0C1FE206802F059FE40
:100BB0006068411C02D0002102F040FE2968A06953
:100BC000C1F82405607D217D2A680843C2F86C05C0
:100BD000D4E900122868C0F80C15C0F81425207D4F
:100BE000012814D1A068411C02D0002102F026FE89
:100BF000E068411C04D002F099FEE06802F031FE8A
:100C0000D4E902122868C0F80825C0F8101570BD94
:100C1000084908B5085C0090684602F045FED0F827
:100C200010050099C84010F0010000D0012080F0AC
:100C3000010008BDE87200002DE9FC410646C0072E
:100C40004FF000050ED0104F00240122385D0095B2
:100C500000231146019502F08BFD641C042CF4D393
:100C600000F01CF8B0070DD5074E0024361D0022F9
:100C7000305D032300951146019502F079FD641C57
:100C8000042CF4D3BDE8FC81E47200000249085C46
:100C9000012102F055BE0000E472000010B50024EE
:100CA0002046FFF7F3FF641C042CF9D310BD042881
:100CB00001D2FFF7ADBF0020704710B50024FFF749
:100CC000BBFF204610BD00002DE9F0470546861CFD
:100CD00090460F464FF001090020FFF70CFF1B4C18
:100CE00020683860D4E90001401AA16804F21C476A
:100CF000081A0EE00121384602F0A2F801F058FE71
:100D00000146384602F09CF8D4E90001401AA16877
:100D1000081A401C8642EDD8B8F1000F03D0052018
:100D200065F3891002E0062065F39F50A2682168F0
:100D3000114004EB8101C86020683044206000202D
:100D4000FFF7DBFE4846BDE8F087000054040020B2
:100D500030B482680468531C8360A154D0E9011246
:100D60008A4202D330BC02F00ABC30BC704700009B
:100D7000034803C8814201D1012070470020704719
:100D8000540400200249084490F9300070470000E4
:100D90008C0100202DE9F05F26484168F1B3DFF8AF
:100DA00098B00E688146DBF8004087688078E11BC8
:100DB00021F07F45ED1CB0B9DFF880804FF4803022
:100DC000C8F84403C8F804031120FFF7EDFB112015
:100DD000FFF721FC4FF0010AC8F800A02F2005F012
:100DE0001FFC89F802A0B54200D23546124BE81923
:100DF0003C3320F07F401860DBF800105A46091B96
:100E000021F07F41001B20F07F40C91C81420FD997
:100E1000106818602F2005F003FC00E004E0BDE836
:100E2000F05F1120FFF70DBCBDE8F05F05F0FABEE2
:100E3000BDE8F09F2800002004150140001001408B
:100E400010B50021024802F006F880F3100010BD32
:100E5000700800200E4910B50A784C780023A24291
:100E600012D0521CD2B20A70022A00D10B70084A6A
:100E70000B780C3252F8232002608868104420F06E
:100E80007F408860012010BD0360002010BD00007D
:100E90002800002002490A88028089788170704702
:100EA000447300002DE9F0418AB0202700260997FD
:100EB00002F072FE054602F087FE804602F0EAFF6D
:100EC000C82002F075FF052002F0AAFF002002F002
:100ED00033FE02F0E1FD00208DF8200004460022E0
:100EE000012108A801F052FB30B1002002F0E0FF20
:100EF000641CE4B2642CF2D3C82001F019F901207B
:100F00008DF820000146002208A801F03FFB08B33D
:100F10001E480078F0B1002002F040FE00281DDDE0
:100F200009AA69460020099702F0D0FDB0B19DF8EA
:100F30000000082812D11548DDF801100C38C0F85F
:100F400003100DF1010001F083FB002001F02AFAEB
:100F5000012603E04FF4967001F0EAF84FF4AF7009
:100F600001F0E6F802F096FF002002F0E5FD002017
:100F700002F0F2FD284602F01BFF404602F050FF4F
:100F800002F08AFD0AB03046BDE8F081C6000020BC
:100F9000002207E010F8013BFF2B01D00020704732
:100FA000521CD2B28A42F5D30120704770B50C466C
:100FB00005460D2910D801F077F808B1012070BD61
:100FC0000648007840B901F0ABF928B1214628461F
:100FD000BDE8704001F068B8002070BDBA00002084
:100FE0000149087070470000B400002001460D223E
:100FF0000148FFF797B900009808002001F012BFE0
:10100000FFFFFFFFFFFFFFFFFFFFFFFFFFFFFFFFF0
:10101000FFFFFFFFFFFFFFFFFFFFFFFFFFFFFFFFE0
:10102000FFFFFFFFFFFFFFFFFFFFFFFFFFFFFFFFD0
:10103000FFFFFFFFFFFFFFFFFFFFFFFFFFFFFFFFC0
:10200000F0B50746204889B0154600780E4698B1CD
:10201000012814D0022834D110221C4904A8FEF74C
:1020200081F91B490D2204A8FEF77CF90024164A09
:102030006846521C21460DE010221449F3E7102295
:10204000124904A8FEF76EF904A800F0B7F8EDE70E
:10205000052C02D2135D035500E00155641CE4B267
:10206000102CF5D301F06EF804A801F07DF8694654
:10207000084601F03DF82B466A463146384600F0E6
:1020800047FB09B0F0BD0000B4000020477300001A
:102090009808002003490268C1F8012000794871BE
:1020A00070470000B4000020F0B50746081D89B055
:1020B000C6B206208DF8100004AC0D46601CFEF779
:1020C000E9FE2A463946201DFEF72CF9174D2878DF
:1020D00008B1002000E00220FEF782FF701EC2B2AD
:1020E000611C601CFFF78CFF01200090002301AAF7
:1020F000314604A800F060FA18B99DF804000B28D6
:1021000002D0002009B0F0BD01AC0322A01DA11D2A
:10211000FFF776FFA01D00F0EFFA0028F2D0287834
:1021200010B9601CFFF7B6FF0120EBE7BA000020F2
:1021300010B5044601F046FD6043400004D0034959
:10214000BDE810408001084710BD00006173000029
:10215000014803F0F3BF000000100000F0B54E236B
:10216000B3FBF2F5022303704F23841804F8013CFB
:1021700081B10123541E0BE003F003068E5DB6FB14
:10218000F5F705FB176605FB0366C6545B1CDBB25F
:10219000A342F1DB01210DE04318445C13F8013C3C
:1021A000E31ADBB2052B03D2C3F1050323444354E6
:1021B000491CC9B29142EFD3F0BD00000349D1F8E8
:1021C00007200260C97A017170470000BA00002040
:1021D000F0B52F4D87B000262878012701ACB0B1AB
:1021E00003208DF80400601CFEF754FE0020FEF76B
:1021F000F7FE0322611C601CFFF702FF002303AA05
:10220000042101A8009700F0D7F9A0B117E002203F
:102210008DF804000521601C00F086F901220621DA
:1022200001A800F0B3F950B1601CFFF733FF2F7025
:10223000002007B0F0BD9DF80C00092802D02E70D8
:102240000320F6E703AC0922601C611CFFF7D8FEEF
:10225000601C00F051FAC0B19DF8100020B10128B7
:1022600005D0022800D12E709DF81000E1E7601D16
:1022700000F076F90D21074800F056F90548FEF701
:10228000B5FE012000F08EF8EDE72E700220D0E7B9
:10229000BA000020A508002041F6FF700078FF2852
:1022A00001D0012070470020704740F6817041F254
:1022B0007E01095CFF2905D00F20B0EB111F07D06C
:1022C00008097047401E00B20028F0DA0E2070475F
:1022D00001F00F00704700003EB5104C0020207048
:1022E000FFF7DAFF98B94FF4805090F87E00FF288E
:1022F0000DD0FFF7DAFF01460E2808D2684600F03D
:1023000046F80098C4F8030001A800F029F9BDE8D8
:102310003E400248C01C00F09BB90000BA000020FB
:1023200010B58AB004208DF8040001200146009009
:10233000002306AA01A800F03FF930BB9DF8180061
:102340000A2822D10DF11900FFF7A4FE05208DF80F
:10235000040001AC601CFEF79DFD0D21201D00F066
:10236000E3F8201DFEF742FE0120FEF739FE1022A1
:10237000611C601CFFF744FE0122112101A800F03E
:1023800005F910B101200AB010BD0020FBE701EBF8
:10239000C10101F580510A6802604A684260097A09
:1023A000017270472DE9FE4300265E4FB046344669
:1023B00000285ED00025E94629466846FFF7E7FF7A
:1023C00058490422C91C6846FDF7D7FF38B955495A
:1023D0000522C91D09F10400FDF7CFFF80B16D1C76
:1023E000EDB20E2DE8D3002529466846FFF7CFFF52
:1023F0004C490422C91C6846FDF7BFFF10B10CE030
:102400002C4632E0052109F10400FEF7C1FD20B1A0
:10241000D7F807000190F87A13E06D1CEDB20E2D8D
:10242000E2D3002529466846FFF7B1FF0921684637
:10243000FEF7AEFD48B157F8030F009078680190A1
:10244000387A8DF808002C4631E06D1CEDB20E2D67
:10245000E8D3B8F1000F07D004EBC40069460922A5
:1024600000F5805003F0A4FE3EB3FFF715FF28B33C
:1024700056E0002421466846FFF789FF29490422D7
:10248000C91C6846FDF779FF0028EED0641CE4B251
:102490000E2CEFD3002421466846FFF778FF042175
:1024A0006846FEF775FD20B1D7F8030000900126BD
:1024B000D2E7641CE4B20E2CEDD331E0FFF7F5FE59
:1024C000A0422DD00E2C2BD04FF48051002040F68E
:1024D00081720F2591F87E10531C04E041F27E01B9
:1024E0009042095C0DD0CE43360706D0B5EB111FE4
:1024F0000AD164F31F11C9B20AE001F0F0012143CF
:1025000006E044F0E00103E0401C00B29842E5DB45
:1025100041F27E02104403F029FE0120BDE8FE8353
:102520000020FBE7BA000020F0B50B4B0025C3F8F4
:10253000005101241C602A46084E09E0D3F80071BE
:10254000002FFBD037688754C3F80051521CD2B219
:102550008A42F3D35C60F0BD00D0004008D5004053
:1025600003490268C1F807200079C872704700006B
:10257000BA00002010B5044601F066FA00E030BF52
:1025800001F01AFBB0EB440FF9D310BD10B5094CA4
:10259000134600226270A2700A460146184601F0F6
:1025A0000BFA08B910BD30BF60780028FBD0A078C6
:1025B00010BD0000BA0000202DE9FC4780460A202B
:1025C0000A9D009016460F46284601F071FC012432
:1025D00001F054FA01F05EFB0028FBD101F0EAFAA9
:1025E00081461E2001F0FCFB01F056FA2A463946CE
:1025F0004046FFF7CBFFE0B10224284601F058FC2B
:1026000007208DF804000A20FFF7B4FF2A460121B5
:1026100001A8FFF7BBFF60B1284601F0BFFA40B147
:10262000202000906A463146284601F04FFA00B15A
:10263000002401F023FA00BF01F02CFB0028FBD19D
:10264000484601F0CDFB01F027FA2046BDE8FC87A3
:102650002DE9FF41054601F01DFB264C0646EDB372
:1026600028786978EA7800EB0120A978090401EB61
:102670000261471801F00EFC204601F027FB50B123
:102680000021084601F00EFB28B1384601F02EFB70
:1026900008B1012402E0012407E037B121460846D1
:1026A00001F000FB08B1012700E00027641CE4B240
:1026B000082CF2D301F064FA0446C2B229466846F7
:1026C000FFF74CFD87B12146684601F01FFB58B16A
:1026D0000120002E05D001F0DFF900E007E030B165
:1026E000012004B0BDE8F0810020002EF9D00020C8
:1026F000F7E700000406080A10B503220349FDF7B6
:102700003CFE08B1002010BD012010BD4473000044
:1027100070B5002409E000BF11F8015B12F8016BED
:102720007540641C00F8015BE4B29C42F4D370BDB8
:102730000278521C027002788A4201D30021017093
:10274000704700002DE9FC5F0E008346DDE90C4771
:10275000C6F1000098469246814600D408460125FD
:1027600003E000BF90FBFAF06D1C5045FADAA84573
:1027700000D9454624B1002E01DB780700D5641E40
:10278000B80702D5B8F1000F0AD0F80708D13CB15C
:10279000A54205D220215846641EFEF7D9FAF6E775
:1027A000002E02DA4E462D2102E0780703D52B21B8
:1027B0005846FEF7CDFA07F0030002280BD1B8F116
:1027C000000F08D13CB1A54205D230215846641E05
:1027D000FEF7BEFAF6E7CDE90047434652463146DA
:1027E000584604F025FDBDE8FC9F000070B50D467D
:1027F000044600684FF4887103F00CFF4FF49071A9
:10280000206803F007FF4FF49271206803F002FF85
:102810004FF4A271206803F0FDFE20681249C0F851
:10282000041320686907000B40B2090E002806DA7D
:1028300000F00F0000F1E02080F8141D03E000F12B
:10284000E02080F8001420680121000B40B200F065
:102850001F0291404009800000F1E020C0F8801282
:10286000C0F8001170BD00001003020002460020F5
:102870001268930702D0530702D47047500714D54B
:1028800002F00300012802D002280CD105E0C2F3B7
:1028900083100B68801C184404E00223086803EBD3
:1028A00092521044086001207047086800EB925370
:1028B000C2F38910401CEEE72DE9F047394E00279E
:1028C00080463D46DFF8E090D6F804A057E003D0FC
:1028D0000446D0F81C8035E099F8002002EB420154
:1028E000521CD2B289F8002009EBC10199F80230DC
:1028F000091D9A4201D189F8005048680A780446B7
:10290000012A12D0022A02D0032A3BD108E004F0A7
:102910009BFA00B10127257434E00574C06900E01A
:1029200070680028F9D170602CE0207C50BB88686A
:102930006060C868A0600869E0604869A061F078DC
:1029400000B165606268B168184B501A20F07F4092
:10295000984202D2A168084406E0881AA16820F0D3
:102960007F40814202D9081A206000E0256065603E
:102970000120A56020742046E56104F047FAB8F113
:102980000000A4D199F8001099F801008142A3D168
:1029900017B97168514502D00120BDE8F0870020C9
:1029A000FBE700002800002048020020FFFF7F0016
:1029B0002DE9FF410026234800F03FFA2148001F7F
:1029C000074600F03AFA204C60680090A56800E0E5
:1029D00000986946284004EB80000C30FFF746FF62
:1029E0000028F5D101AA009901EA050304EB83034D
:1029F000491CDB6842F82030401C00910228F2D3C9
:102A0000019800F0030001280BD0022810D1019892
:102A1000032101EB90500099BDF80A6001EB900092
:102A200005E00198BDF80A60C0F3831008440090E7
:102A3000384600F0FFF908B10098606004B03046F5
:102A4000BDE8F0816C080020540400204FF000091C
:102A500088B04E464FF0040849460220FEF72DF993
:102A600008B1FEF73DF84FF40041002003F0E0F913
:102A700008B1FEF735F803F067F8002001F0C6F85A
:102A800028B901F083F800F50340FEF729F84B2040
:102A900001F08EF94FF4FC7001F0B2F928B901F0A1
:102AA00075F800F50340FEF71BF8FFF751FBFFF741
:102AB00013FC00F0F1FF28B901F068F800F50340BD
:102AC000FEF70EF8DFF8C4A00321BAF8000001EB0E
:102AD00000402FA103F052F95FF0010503F042F826
:102AE0000028FBD100273C462046FEF7E0F818B14D
:102AF00005FA04F03843C7B2641C042CF4D3F8433D
:102B00008DF8000026B10D216846FEF74FFA11E05E
:102B100001F0E6F901F0EAF911226946022000F01D
:102B20004BFF08B908E030BF01F0E6F90028FAD001
:102B300001F0E8F981460BE0BAF8000022A105EBAC
:102B4000004003F01BF900BF03F00CF80028FBD194
:102B500086F00106B9F1000F10D1BAF800001EA1ED
:102B600005EB004003F00AF902F0FCFF0028FBD15E
:102B7000FEF798F910B1FFF72BFB8046B8F1000F74
:102B8000B0D1FFF725FB8046ACE7000058010020DC
:102B900047617A656C6C2064796E616D6963207041
:102BA000616972696E67206578616D706C6520730C
:102BB0007461727465642E20446576696365206D66
:102BC0006F64652E000000005458206669666F200F
:102BD0006572726F7220000047617A656C6C653AAD
:102BE000207472616E736D697373696F6E206661B4
:102BF000696C6564000000002DE9F047C788044651
:102C0000181D16468946B0FBF7F1B0FBF7F207FB3B
:102C100012009A193A44D21CB2FBF7F2DDF820A058
:102C200001E02468491E0029FBD13D1A8846B542BF
:102C300016D818E0BAF1000F05D0211809EB0800EA
:102C40002A46091D04E0204409EB08012A46001D1C
:102C5000FDF768FB00202468761BA844B74201D921
:102C6000354600E03D46002EE4D1BDE8F087000087
:102C700030B5024659B103F007F90021074C09E0CD
:102C800004EB810315685B88AB4202D11160002020
:102C900030BD491C8142F3D3052030BD44010020E2
:102CA0002DE9F0415C4903780446D1E9030200258F
:102CB000082B77D2DFE803F0042B4877726E8795F4
:102CC000217C914208D238B100EB81018A6C521C00
:102CD0008A640168491C0160A17B2E4661F30706E6
:102CE0002189677B61F31F466189606861F30F0585
:102CF000217B61F31745E17B61F31F6501F020FD46
:102D00002A4631463846BDE8F04100F0ADBE48697C
:102D1000407D10B94148FEF771F92F46218965F3CE
:102D2000070761F31F476189267B61F30F05617B0C
:102D3000606861F31F6501F003FD2A46394630469D
:102D4000BDE8F04100F086BE217B914208D238B147
:102D500000EB81018A6C521C8A640168491C016085
:102D6000A07A217A60F3070561F30F25E17A667A8C
:102D7000676861F3174538B11FB928482630FEF758
:102D80003DF9384601F0DCFC29463046BDE8F0410B
:102D900000F03BBFBDE8F04100F07CBE00F080FFDA
:102DA000BDE8F08131E01E484168491C416001786E
:102DB0000029F5D0816811B1491E8160F0E7BDE8B6
:102DC000F04100F05BBEA379934208D238B100EB2A
:102DD000830293685B1C93604268521C42608A685D
:102DE0000CE0A379934208D238B100EB83029368D8
:102DF0005B1C93604268521C42604A68002ACFD034
:102E000061792079BDE8F0411047BDE8F041034801
:102E10007F30FEF7F3B80000D40000203D04050029
:102E2000B408002002490F220A7088617047000030
:102E3000D4000020002100F009B8012100F010B8F2
:102E400008B56A46FDF719FA009808BD08B56A4644
:102E5000FDF7F9F908BD08B56A46FDF7DBF908BDCD
:102E600008B56A46FDF7E2F9009808BD08B56A465C
:102E7000FDF710FA009808BD70B5044600252846F5
:102E8000FDF739FE21686268086890420ED9401E3D
:102E900008600178A38AE26801FB0325227A216891
:102EA000101AC0B20A79824200D208710020FDF7E0
:102EB00024FE284670BD70B505460C460020FDF77F
:102EC0001AFEE868A98A201AB0FBF1F12A68106896
:102ED000431C13600170BDE870400020FDF70DBE7B
:102EE00010B530B1017A42680368891AC9B21A6014
:102EF00006E00E2010BD03681A68541C1C60117097
:102F0000491EC9B2F7D2006800210171084610BD00
:102F1000C20800F007030120895C98400840704710
:102F200010B5C20800F00703885C01249C402043D0
:102F3000885410BD70B5074C251F20682968496862
:102F4000884202D30448FEF759F82868216880684F
:102F5000405C70BD10010020440001000148006881
:102F6000704700001001002010B5044605480068B5
:102F70004068A04202D80448FEF740F80148001D0E
:102F8000046010BD0C0100204C00010001484068A5
:102F9000704700001001002010B504460548006885
:102FA0000068A04202D80448FEF728F80148001D36
:102FB000446010BD0C0100205800010010B5040051
:102FC00002D10548FEF71AF8044800210460001DEC
:102FD0000160416010BD0000270001000C010020CD
:102FE0000948021F4168491C4160126813689942F0
:102FF00008D3002343600168491C01605268914274
:1030000000D303607047000010010020002839D071
:10301000401E00BF00BF00BF00BF00BF00BF00BF19
:1030200000BF00BF00BF00BF00BF00BF00BF00BFA8
:1030300000BF00BF00BF00BF00BF00BF00BF00BF98
:1030400000BF00BF00BF00BF00BF00BF00BF00BF88
:1030500000BF00BF00BF00BF00BF00BF00BF00BF78
:1030600000BF00BF00BF00BF00BF00BF00BF00BF68
:1030700000BF00BF00BF00BF00BF00BF00BF00BF58
:1030800000BFC5D170470000F0B50546047815486B
:1030900089B0164640F82420124A08690832A2F185
:1030A0000C0742F82400487F385520226846FDF777
:1030B00039F904942878385C48B10EB10A4A00E026
:1030C00000226946281D03F013FC09B0F0BD0EB1C3
:1030D000064A00E00022694605F10C0003F0DAFA26
:1030E000F3E70000040000200D710000596F00009C
:1030F00070B5124D06464FF080746868814202D068
:103100001022FDF70FF90E490020C1F8000101223D
:103110000A6001E0641E0ED0D1F80021002AF9D027
:10312000C1F80001A9688E4203D010223046FDF795
:10313000F9F8012070BD002070BD000014000020CF
:1031400000E000400549064801F11002C0E9001204
:103150001032826003480160012070475C0100204A
:103160001400002004E500400146024810220068D7
:10317000FDF7D8B8140000202DE9F04104461028CE
:1031800002D30B48FDF73AFF094E0A4D761D204643
:1031900000F07EF8070008D0AF4202D13046FDF7BC
:1031A0002DFF384600F03AF8F1E7BDE8F081000065
:1031B000D0000300ADDEADDE0148006870470000BE
:1031C0004001002010B50020114A014600EB4003E9
:1031D0009C186170A170D154401CC0B21028F5D366
:1031E000DE22CC210B48FDF7AFF80A4A0020A2F1FD
:1031F000180100BF00EB001302EB430341F820303D
:10320000401CC0B20628F5D303490620086010BD53
:10321000A80A0020B00B00204001002070B5104C1F
:1032200006462068062802D30E48FDF7E7FE304622
:10323000FDF7A6FB18B90B48401CFDF7DFFE0A4D51
:1032400020680A4955F82000884203D00548801CB0
:10325000FDF7D4FE216845F82160491C216070BD4E
:103260004001002080000300980B0020ADDEADDEA1
:1032700010B50446102802D30348FDF7BFFE0349EA
:1032800004EB4400085C10BDC2000300A80A002043
:1032900070B500260446102802D30C48FDF7AEFE98
:1032A0000B4D04EB4404285D70B105F1300000EBD8
:1032B0008401601910F8022F51F822600321FFF7F2
:1032C00037FA285D401E2855304670BDA200030025
:1032D000A80A002070B50C460646102902D31248F1
:1032E000FDF78CFE3046FDF74BFB18B90E48401C2D
:1032F000FDF784FE0D4D04EB4404285D032810D235
:1033000005F1300000EB8401601910F8012F41F83D
:1033100022600321FFF70CFA285D401C285501208C
:1033200070BD002070BD00008C000300A80A0020C2
:1033300010B50446102802D30948FDF75FFE09497D
:1033400004EB44000A5C42B101F1300202EB80025E
:103350000844807852F8200010BD002010BD000005
:10336000B3000300A80A00200B4810B50168002430
:1033700079B10A4A0A4B02EB8102491E52F8044D08
:10338000136001602046FDF7FBFA10B90548FDF710
:1033900035FE204610BD000040010020980B0020A3
:1033A000ADDEADDE7800030000487047408100408C
:1033B0002DE9F74F904607004FF0000502D1344841
:1033C000FDF71CFE334C4FF4803BC4F808B3324E7B
:1033D000B07818B12E48801DFDF710FE706818B146
:1033E0002B480930FDF70AFEDFF8B0A077605FEAEE
:1033F00008004FF000094FF00108AAF1040724D09B
:1034000001282FD0022829D021481D30FDF7F6FDD4
:1034100086F80280C4F840910199294489B2396044
:103420003F68C4F84480DAF80060D4F8400118B16D
:1034300017482B30FDF7E2FDAF4215D3AE4201D362
:10344000BE4221D3124833301CE0C4F84480DAF87D
:103450000050C4F84080C4F84091D9E70F48001DDF
:103460000568D5E73D68D3E7BE4201D2012000E000
:103470000020B54201D8012100E00021884203D19B
:1034800003483E30FDF7BAFDC4F804B3BDE8FE8F33
:1034900086000400008000401801002044850040A0
:1034A000004870474880004070B5144C01266660A3
:1034B000E660666412480025056011483C300068EB
:1034C00010B11048FDF79AFD4FF0FF30C4F8080323
:1034D000C4F840510A490420083108600A48456090
:1034E0000670457085700820FDF774F84FF0E021F4
:1034F0004FF48070C1F8000170BD000000800040F2
:1035000008850040470004001801002001480078A9
:10351000704700001801002003490120086003499A
:103520000020087070470000008000401801002053
:1035300070B5074801250561C560064C00260820C6
:1035400066606670FDF746F8A670257070BD0000D5
:1035500000800040180100200148407870470000BA
:10356000180100200FB408B50399002904D004AA5B
:1035700000926A4600F00FF801B05DF814FB10B538
:1035800082680446002A05D0D4E9040321689847DC
:103590000020A06010BD2DE9FC4791460C0080463C
:1035A00076D014F8011B39B125290ED04046FDF71D
:1035B000CFFB20780028F4D198F80C00002867D0C1
:1035C0004046BDE8FC47FFF7DABF00200122217822
:1035D0002B291BD02D2902D0302908D102E040F040
:1035E000010001E040F00200641C002AEFD1002538
:1035F0002A290ED02178A1F130020A2A11D205EB36
:10360000850201EB4205641C303DF1E740F0040007
:10361000EAE7D9F800100B1DC9F800300968641CEE
:103620000D44217800232E290BD114F8011FA1F19C
:1036300030020A2A05D203EB830201EB4203303B3E
:10364000F3E76C290DD068290BD0692921D00BDC58
:10365000252918D0582931D063290ED0642915D1D5
:1036600017E014F8011FECE7702969D0732932D0F4
:1036700075291BD0782909D120E0D9F80000011D57
:10368000C9F8001001784046FDF762FB641C90E722
:103690006CE0D9F800100A1DC9F800200968CDE9CE
:1036A00000500A224046FFF74DF8EFE7D9F8001026
:1036B0000A1DC9F8002009680A2206E0D9F800109E
:1036C0000A1DC9F8002009681022CDE900504046C3
:1036D00003F0AEFDDAE7D9F8001000270A1DC9F89B
:1036E00000200E68C00705D112E04046761C7F1C02
:1036F000FDF72EFB31780029F7D104E02021404668
:103700006D1EFDF725FBBD42C0D9002DF6D1BDE7EA
:103710004EB13046FCF72AFE074604E02021404621
:103720006D1EFDF715FBBD4206D9002DF6D103E055
:103730004046761CFDF70CFB31780029F8D1A5E74F
:10374000D9F80000011DC9F8001005683021404675
:10375000FDF7FEFA78214046FDF7FAFA082000212D
:10376000CDE90001034610222946B0E7BDE8FC87F9
:103770002DE9FF411C46DDE90A7815460E466846EC
:1037800000F092F846EA450141EA840141EA072245
:1037900042EA0841009A00EB8200C0F80017BDE839
:1037A000FF812DE9FF411C46DDE90A7815460E46EA
:1037B000684600F095F846EA450141EA840141EA8D
:1037C000072242EA0841009A00EB8200C0F8001785
:1037D000BDE8FF812DE9FF411C46DDE90A78154669
:1037E0000E46684600F08AF846EA450141EA84013F
:1037F00041EA072242EA0841009A00EB8200C0F841
:103800000017BDE8FF811CB5002100910B46012285
:103810000191FFF7C6FF1CBD1CB5002100910B46AE
:1038200001220191FFF7D6FF1CBD1CB500220B46FB
:10383000009211460192FFF7B4FF1CBD1CB5002297
:103840000B46009211460192FFF7C4FF1CBD1CB548
:10385000002100910B46012201911146FFF7A1FFC3
:103860001CBD1CB5002100910B460122019111469F
:10387000FFF7B0FF1CBD13B50C46684600F022F8F8
:10388000009900EB8101D1F8002722F44032C1F801
:103890000027009900EB8100D0F8001741EA0441AD
:1038A000C0F800171CBD00000168202902D24FF0AB
:1038B000A040704701F01F010160014870470000FF
:1038C000000300500168202902D24FF0A040704749
:1038D00001F01F0101600148704700000003005023
:1038E0000168202902D24FF0A040704701F01F016B
:1038F0000160014870470000000300500168202962
:1039000002D24FF0A040704701F01F010160014852
:10391000704700000003005001B56846FFF7E0FF64
:10392000009A01219140C0F8081508BD01B568460C
:10393000FFF7E4FF009A01219140C0F8081508BD87
:1039400038B501240090684631B1FFF7ADFF00990A
:103950008C40C0F8084538BDFFF7A6FF00998C40A1
:10396000C0F80C4538BD00001CB5094C0144D4E931
:103970000034CDE900346C4606E000BF54F8203036
:10398000D3F81035401C08C28142F7D81CBD000096
:10399000EC720000034908B508440021016000688A
:1039A000009008BD0060004002494058012800D046
:1039B00000207047006000402DE9F041204D164680
:1039C00088460746082801D3042035E0B8F1000FE7
:1039D00003D0202E03D906202EE003202CE0384609
:1039E00001F06EFA032801D3092025E0384600F0E3
:1039F000FBFF032801D30A201EE000F01BFD022874
:103A000001D2082018E000F0A5FE044606704078B8
:103A1000324640F0010060704146A01CFCF782FC79
:103A2000F8B2214601F04EFA10B10120BDE8F08154
:103A30000448FDF7E3FA0F2028700020F6E70000A5
:103A4000D4000020FC0005000149002048607047B8
:103A5000B40800200348C1600261012141700021C7
:103A600081707047BA0000200348C16002610121E3
:103A70004170817070470000BA00002010B500F05E
:103A80009DFD18B1BDE8104000F004B8BDE810403D
:103A900000F092BC7047000010B50B4C606928B173
:103AA00000F042FB0004000C02D005E0022008E018
:103AB000002000F059FE18B100F092FC012010BD6A
:103AC00011202070002010BDD40000202DE9F0410D
:103AD00016460F46044600F087FF154D48B157B112
:103AE000204600F08DFF00783168814205D2062023
:103AF0001AE00B2018E0032016E0204600F076FFC5
:103B000004000DD0A01C0BD02278A11C38463260D6
:103B1000FCF708FC204600F013FE0120BDE8F08110
:103B20000448FDF76BFA0F2028700020F6E700002C
:103B3000D40000202601050010B5082804D305494B
:103B400004200870002010BDC0B200F043FF012027
:103B500010BD0000D4000020084910B54A69527D0C
:103B60000AB10C2002E0082803D3042008700020CA
:103B700010BDC0B201F08CF9012010BDD4000020AE
:103B80000148006970470000D40000200148007817
:103B900070470000D400002000F01ABD082804D3AC
:103BA000034904200870401F704700F01DBF00004B
:103BB000D400002001F092B801484068704700002E
:103BC000B408002001F0A2B810B5012401F094F966
:103BD000F02815D005DCB0B1042809D0EC2812D1AA
:103BE00010E0F4280AD0F82806D0FC280BD101E018
:103BF000002408E0022406E0032404E0042402E098
:103C0000052400E00624204610BD70472DE9F04150
:103C10001D4D064600241D482C70AC6104604460B4
:103C200084601B4800F028FC686140B3042000F069
:103C300099FA05F11C00296900F068F8074630463A
:103C400000F0B8F800EA0706002000F099F80640F6
:103C5000012000F0E5F80640022000F079F8064067
:103C6000002000F0FFF80640012000F0A1FE002037
:103C7000EC6000F05FFD16B10120BDE8F08101208D
:103C800028700020F9E70000D4000020B4080020CC
:103C9000A12C000001484069407D7047D4000020FD
:103CA00070470000084A10B553695B7D0BB10220D4
:103CB00002E0082803D304201070002010BD00F09B
:103CC00063FD012010BD0000D4000020064910B59E
:103CD0004A69527D1AB102200870002010BD00F020
:103CE00029FA012010BD0000D4000020064910B5BB
:103CF0004A69527D1AB102200870002010BD00F000
:103D000025FA012010BD0000D400002010B50F4C92
:103D10006269527D0AB1022014E010290FD871B1F6
:103D200078B10A462161014608481C30FCF7FAFACE
:103D3000064821691C3000F029FA012010BD072037
:103D400000E003202070002010BD0000D4000020FF
:103D50000A4910B54B69024601205B7D0BB1022078
:103D600004E0012A05D0022A04D00E2008700020A9
:103D700010BD002000F088FA012010BDD400002002
:103D80000A4910B54B69024600205B7D0BB1022049
:103D900003E032B1012A03D00E200870002010BDCC
:103DA000012000F0EDF9012010BD0000D40000203A
:103DB00000F014BC10B540B1012808D002280BD087
:103DC000064905200870002010BD012000E00220F7
:103DD00000F00AFC012010BD0020F9E7D40000200B
:103DE000064910B54A69527D1AB1022008700020B8
:103DF00010BD00F079FF012010BD0000D4000020AC
:103E0000064910B54A69527D1AB102200870002097
:103E100010BD00F081FF012010BD0000D400002083
:103E2000014610B50020072914D2DFE801F0040F85
:103E300006080A0C0E00042008E0FC2006E0F8202A
:103E400004E0F42002E0F02000E0EC2001F05AF859
:103E5000012010BD02490E200870002010BD000096
:103E6000D40000200A4910B54B69024600205B7D52
:103E70000BB1022003E032B1012A03D00E200870FA
:103E8000002010BD012001F047F8012010BD000006
:103E9000D400002010B5FFF7FDFE002806D0FFF784
:103EA000EDFD30BFFFF7F6FE0028FBD110BD00008E
:103EB00038B50446012181F31088202505E06A46C3
:103EC000064920460095FFF701FE2046FFF766FEF3
:103ED0000028F4DC002080F3108838BD780800202A
:103EE0000149002048707047BA00002001490020B5
:103EF00088707047BA000020014840787047000081
:103F0000BA0000200148807870470000BA00002005
:103F100010B501F0F3F90349002008610249087067
:103F200010BD00000C090020000100202DE9FE4317
:103F30004D4800684D4C012802D04D48006828B912
:103F400060680078202801D8012100E00021494E56
:103F500003204FF0000830704348C4F80080083058
:103F60000568424F183F89B3006841490839086025
:103F700002A8CDE900043C480C3002680123294620
:103F8000184602F067F910B3012805D0022821D0A5
:103F9000032855D0384851E0029818B136481C38EB
:103FA000FDF72CF8284602F0B8FA18B932481B3849
:103FB000FDF724F801F0D6F9B97D0023CDE9000121
:103FC0007068EAB290F9161018461CE01EE02A4804
:103FD000113833E0029818B927480D38FDF70EF86C
:103FE000284602F09AFA18B923480C38FDF706F86B
:103FF00001F0B8F9B97DEAB2CDE90001706801239A
:1040000090F91610029800F07DFB19E000F072FEA6
:1040100030B101F0A7F90146BA7DE8B200F044FBE7
:104020000023CDF800801A4619461846CDF80480C2
:1040300002F010F9042803D00F480F30FCF7DEFF20
:10404000206838B1012060750C4820610420307070
:10405000BDE8FE8301F052F984F81580C4F81080A1
:1040600000F00EF8F4E70000001400400C090020F6
:1040700034150040000100204406090019410000E9
:1040800070B5FFF745FF1F4D012028701E480168DD
:104090001E4A21F0FF0112691143016002F046FA45
:1040A0001A4C4C3410B302F041FA032802D01848DD
:1040B000FCF7A4FF022001F05FFB002001F0B4FB3D
:1040C00002F034FA032803D011480830FCF796FFB9
:1040D0002878012803D00E480E30FCF78FFF02200D
:1040E0002870002020610B48E06070BD02F012F8DB
:1040F0000228DFD302F040F960600028DAD10448DA
:10410000401FD5E70001002030150040C008002006
:10411000F40509002D3F0000024905200870FFF753
:10412000AFBF0000000100200148006A7047000096
:10413000C0080020034910B5086200F0ADFD024937
:10414000086010BDC00800201C150040034910B5D0
:10415000486200F0A1FD0249086010BDC0080020BF
:10416000201500400449487704490A6822F4E022F7
:1041700042EA004008607047C0080020181500405F
:104180000149087670470000C008002070B50C0097
:10419000054602D10748FCF731FF1DB90548401C10
:1041A000FCF72CFF0448C0E90145BDE87040002041
:1041B000FEF7DABEB30309002409002010B500F0B1
:1041C00099FD044901F1640208B1C86800E08868FB
:1041D000106010BDC00800201CB510494FF440709D
:1041E000086002F0A3F9012812D0022810D0032899
:1041F00013D100200090034602460146019002F0D0
:1042000029F8042809D0BDE81C400548FCF7F6BE93
:104210000021084602F0CEF8F3E71CBD08F5014086
:1042200048020900144981F8310014490A6822F053
:10423000FF020A6048B1114A0B1D0832012807D05D
:1042400002280ED00E48FCF7D9BE086808607047F7
:10425000086840F001000860FF20106040F207107D
:1042600007E0086840F0020008604FF6FF70106039
:104270000448186070470000C00800203415004052
:104280002E04090021100100044981F8320004497C
:1042900008B1012800D1086070470000C008002064
:1042A000101500402DE9FF413E480068012802D06A
:1042B0003D48006830B93D4840680078202801D862
:1042C000012700E0002700F0F5FB384C0126183CE0
:1042D00000B9266102F02AF9012802D03448FCF71F
:1042E0008DFE344D6868007D18B13148401CFCF7E4
:1042F00085FE01F003F8EFB30121084602F05AF8F9
:1043000020B1012828D0022826D10FE001F02AF898
:10431000064601F067FFC7B201F05EFF8446A07D4C
:104320000021CDE90260CDE900710DE001F01AF83D
:10433000804601F057FFC7B201F04EFFA17DCDE9E5
:104340000076CDE90281844668686289218990F906
:104350001630604600F0B8F9FEF700FEE060134842
:104360004C3840696060FFF729FF04B00020BDE8C9
:10437000F04100E001E0FEF70FBE6E7000F0BAFC05
:1043800000280CD000F0EEFF054601F02BFFA27DC7
:1043900004B02946BDE8F041C0B200F085B9BDE8DF
:1043A000FF81000000140040341500400C0900207B
:1043B000370709000001002010B5012080F31088A4
:1043C0000648417D29B1817819B90121817000F039
:1043D0003FFB002080F3108810BD0000F40800208F
:1043E00070B5124C607D00281ED100F0C3FA04F1B4
:1043F0003005A86810B90E48FCF700FE686818B9C7
:104400000B48401CFCF7FAFD02F0C0F818B1084850
:10441000801DFCF7F3FD002002F0D8F80120607544
:10442000BDE8704000F014BB70BD0000F40800202F
:10443000CE02090001F0E2BE30B50D4D85B0687DB9
:10444000002813D000F042FB00F058FF0024AC70AD
:104450006C7505208DF80000684601F007FE0548E0
:10446000047005B0BDE83040FFF7B6BE05B030BD02
:10447000F4080020000100202DE9F041054601204C
:1044800080F31088484E4FF003080024707086F8BF
:104490000080B470746034817481F46007463461C4
:1044A000347506F118007475046044608460C4605B
:1044B00004610475183084604460FEF7F5FF2846F7
:1044C00001F00EFE01F09CFE002002F071F806F1F2
:1044D0003000FEF773FD00210820FCF7BDF8002135
:1044E0000120FCF7B9F801211520FCF7B5F80120EF
:1044F00000F07AF8A6F13405FF20286104206877DF
:104500002A4929622A49696285F82870022185F8BA
:10451000291085F82A8085F82B00052085F82C00C5
:10452000062085F82D00072085F82E00082085F844
:104530002F0085F8304085F8311085F832706920F9
:1045400045F8140B1E2028604FF4167045F8100C27
:10455000022000F091FC0F2000F094FCEC802F7101
:104560006F712C72204601F043FE7078012802D052
:104570001048FCF743FD3770B47074603481748167
:10458000F46034610C48347574758460447000F0D4
:10459000F1F90820FCF713F81520FCF710F884F364
:1045A00010880148BDE8F081F408002004070A0DD6
:1045B00005080B0E9F020900000100200348407D02
:1045C00008B100207047012070470000F408002067
:1045D0000148408B70470000C00800200149488313
:1045E00070470000C008002010B5012181F3108839
:1045F00007490A78824204D04870487D28B100F00B
:1046000027FA002080F3108810BD00F003F8F8E7C7
:10461000F408002030B5224D85B0287869788842AA
:104620003BD008B900F0A6F9687808B9FFF7D4FDC7
:104630001C480024046000F061FE19481830046032
:10464000446004618460C4602878012802D0022894
:1046500008D015E001F06AFF90B10021084601F092
:10466000A9FE0DE0FFF754FC01F060FF032807D11D
:10467000002300941A4619461846019401F0EAFDF9
:10468000FFF79CFD6878287004208DF800006846CC
:1046900001F0ECFC012005B030BD0020FBE700007C
:1046A000F408002054F5014000B585B006238DF8CC
:1046B00006208DF805108DF804008DF8003068464E
:1046C00001F0D4FC05B000BDF0B585B00DF1280CAB
:1046D0009CE8F0008DF80C308DF80D404FF0000C88
:1046E0000190ADF808108DF80E508DF800C0ADF8AF
:1046F0000A208DF80F608DF81070684601F0B6FC46
:1047000005B0F0BD70B586B00226DDE90A458DF82A
:1047100008108DF8092001908DF80A308DF800609E
:104720008DF80C508DF80B40684601F09FFC06B0E8
:1047300070BD000001498860704700000001002042
:1047400010B5012181F3108801F080FD002080F375
:10475000108810BD10B5012080F3108801F078FD9D
:10476000002181F3108810BD10B50446082802D33B
:104770000348FCF743FC0348204490F8280010BD90
:10478000AD030900C008002070B5082819D20F4AEF
:10479000024482F828108207D40EFF22A240D2439E
:1047A000042801D20A4D01E0094D2D1D2868104052
:1047B0002860084600F05EFA2968A0400843286097
:1047C00070BDBDE870400348FCF718BCC00800206D
:1047D00024150040A703090010B51B4C0020607091
:1047E000FEF7A8FB19490860FEF7B8FB1849887561
:1047F00001F09CFE012807D001F098FE022802D0AB
:104800001448FCF7FBFB002000F0B6FFFEF7CCFDE0
:10481000114908606068091D40680860A0680028A8
:1048200011D0007820B1FEF7BFFDA16800F002FCB6
:10483000A0680179002906D000F0D0FBA068BDE88F
:10484000104000F0D9BB10BD000100200815004049
:10485000F40800209706090050F5014010B501F05A
:104860000FFE002820D0114800210181418101F074
:10487000B9FC0F49086001F0B5FC012181400C48EA
:10488000001D026822F0FF021143016001F0A4FC48
:10489000064C1834206001F099FC60600548E06027
:1048A000BDE81040FFF798BF10BD0000F4080020DD
:1048B0002C150040A542000015480021016001218F
:1048C00001601448016821F480710160016821F0E1
:1048D0000F01891D0160016821F4702141F440310C
:1048E0000160001D016821F000710160016841F064
:1048F00080710160016821F0FF0141F02001016039
:10490000016821F47F4101600120FBF758BE0000DF
:10491000FC1F00401415004070B5134C1348A168EB
:1049200000F096FE6060114C4C3C607FFFF71AFC73
:10493000206AFFF7FFFB606AFFF708FC002560199B
:1049400090F828102846FFF71FFF6D1C082DF6D39E
:10495000074914F8300F08606078FFF763FCA0780F
:10496000BDE87040FFF790BC000100200C0900205A
:104970000C1500400C4910B5002008600A484FF49F
:1049800040744C380460FFF797FFFEF789FD064935
:1049900008310860091F0548086003485038046062
:1049A000BDE81040FFF7B8BF54F5014004110040C6
:1049B00010B504460448406810B90448FCF71EFBD3
:1049C0000348047510BD0000000100206E040900BA
:1049D0000C09002010B5012181F3108801F09AFD27
:1049E000002080F3108810BD01F097BD10B50121A3
:1049F00081F3108801F094FD002181F3108810BD2F
:104A000001F091BD03490122086101460248FEF709
:104A1000CFBC0000F40800209965000070B50C467A
:104A200001F0D4FD074D2869A04202D30648FCF7E7
:104A3000E5FA28690122211A0448FEF7B9FC002092
:104A4000286170BDF4080020D606090099650000B1
:104A500010B5FEF75BFD012822D101F0B1FD10B1C8
:104A60001048FCF7CBFA002264210F48FEF7A0FCA7
:104A70000E48007F80B90E48012101600022000726
:104A8000C0F80021016000BF00BF00BFAFF300808D
:104A9000D0F800110029FBD0BDE81040FEF73CBD66
:104AA00010BD0000B406090099650000C008002090
:104AB00014050040044810B5006918B9FEF74CFD14
:104AC000002800D0012010BDF408002010B5FEF72A
:104AD0001DFD01280ED0FEF72BFD0748007F10B901
:104AE000012081074860002001F070FD024900208C
:104AF0003431486010BD0000C00800200B4810B5DC
:104B00004068407D30B1012000F08EFE08490889E0
:104B1000401C08810749002008600548343803C854
:104B2000BDE81040091A0020FFF778BF00010020FF
:104B3000F408002054F5014070B586B0FFF7BAFFC5
:104B4000494D4A4E05F1340458B100F0BDF8A07843
:104B5000002869D0FEF744FA06B0BDE87040FFF7C0
:104B60006BBC2078012802D0022804D008E000F0B5
:104B700017FF28B170E0307804286DD003286BD07F
:104B8000FEF72EFA00F0A0F8A07868B1FFF754FC09
:104B900001F0C0FA022840D303208DF800006846D7
:104BA00001F064FA06B070BDFFF734FD20B10020BB
:104BB0006968FFF733FFEBE72078F0B1012816D0E2
:104BC000022817D02A48FCF719FA687E0128DFD19D
:104BD00000F090F80028DBD12078D8B1012811D05E
:104BE0000228D5D022481A30FCF708FAD0E700F0A6
:104BF00099F8EAE700F01AF9E7E700206968FFF79B
:104C00000DFFE2E701F092FC0028C1D101F00CFC9D
:104C10000028BDD1FFF75AFFBAE706B01448BDE837
:104C200070403630FCF7EAB92078022808D0FEF749
:104C3000D7F9696806B00020BDE87040FFF7EEBE06
:104C40003078042808D0032806D0FEF7C9F906B04A
:104C5000BDE8704000F0EAB8686806B04008BDE8FA
:104C60007040FFF7CFBE0000C00800200001002008
:104C7000D0040900024610B50020014622FA01F3D3
:104C800003F00103C1F10704A3400343491CC9B267
:104C9000D8B20829F2D310BD2DE9F0410024064610
:104CA00025461827E80026FA00F0C0B2FFF7E2FF19
:104CB000694207EBC101884020436D1CEDB20446F8
:104CC000042DEFD3BDE8F0810348416809B1491EC6
:104CD0004160FFF773BA0000F40800200148406902
:104CE00070470000C008002001494861704700007B
:104CF000C008002004480178022902D0406800283A
:104D000000D0012070470000F408002001484068EE
:104D100070470000C008002001494860704700004B
:104D2000C00800202DE9F04186B000F0E7FA01F05C
:104D3000FDFB3A4D05F1340420B3688BB0B32189F3
:104D400081423BD30121002001F034FB01F044FA01
:104D500026898046648901F045FA074600F002FB87
:104D6000014601208DF80000ADF808608DF80C7048
:104D7000CDF80480ADF80A408DF80D10684601F0BA
:104D800075F944E001F0C6F9022840D3FFF7B2FFFD
:104D900068B1FEF7FBF8D0BB287E20B9FEF7DEF83D
:104DA000E168884233D1FFF759FD30E006E0E06862
:104DB000FEF7DAF80020FEF7EFF8F4E7FEF7CCFB99
:104DC00010B11748FCF71AF9FEF7B4F8154909684D
:104DD000884202D06089401C608113484078A0B9A5
:104DE000FFF788FF88B101F0FDF9064600F0BAFA36
:104DF000A17D8DF806108DF8050007228DF80020A2
:104E00008DF80460684601F031F9FFF7E5FC296888
:104E100006B00120BDE8F041FFF700BEC008002049
:104E20007C050900081500400001002070B5002431
:104E3000FEF780F80D4D2968884207D0FEF77AF812
:104E40002860FEF78BF80A49012488750948641E1A
:104E50000078044201D1FFF713F90548343841685E
:104E6000BDE870400020FFF7D9BD000008150040E4
:104E7000F4080020000100200149C860FFF79EB936
:104E8000C008002001498860FFF798B9C0080020D9
:104E900010B50446012181F310880748017821B13B
:104EA000407D10B10548FCF7A9F8204601F044FB0D
:104EB000002080F3108810BDF4080020680309006A
:104EC00001F043BB10B5012282F3108801F04AFBC8
:104ED00058B10848817819B9407D08B1FFF7B8FD8D
:104EE000002080F31088012010BD002080F310887E
:104EF00010BD0000F4080020014890F83000704711
:104F0000C0080020024981F830000249086070475B
:104F1000C00800200C1500400149087770470000C8
:104F2000C008002070B51149114A0025487802EBED
:104F30000010027B22B10F4AD2F80C2102B10125E8
:104F4000807A0870012000F0DFFB0B4C1DB1A068D7
:104F5000806800B180476068002806D00179002988
:104F600003D0BDE8704000F01BB870BD30090020D0
:104F7000687300000010004020010020074800690D
:104F8000012805D0022805D0032805D100F09AB8E1
:104F900000F04CB900F0E4B8704700003009002080
:104FA000827B002193000B4A1344C3F81019C37B82
:104FB00002EB8302C2F81019427B0121837BC07B84
:104FC00001FA02F201FA03F3814003481A430A434B
:104FD0000260704700F0014008F501404279054B3E
:104FE000C079012103EB80000AB1016670470163BB
:104FF000704700000060004082680021C2F8401144
:10500000C17B094ACB0009490B44C3F81025C37B77
:10501000826801EBC301C1F81425C17B01208840DF
:1050200003490860704700001011004000F0014083
:1050300004F501402DE9F0410746886800260C463A
:10504000C0F840618868097B1A4D00F5A07005EB37
:10505000C101C1F810056278E178207B00F08EFC78
:10506000607B05EBC000C0F81075617BA06805EBA4
:10507000C101C1F814051048C0F80C61C0F81061F6
:10508000A17B0E4805EBC101C1F810056278E178FB
:10509000A07B00F061FC217B0120627B00FA01F122
:1050A00000FA02F21143A27B9040014304480160E0
:1050B000BDE8F08100F00140001000400C110040FC
:1050C00004F501402DE9F0411F4E0220002530700B
:1050D0000320707075603575B0691C4C401CB06160
:1050E000C4F80C51C4F80051C4F81051C4F804516C
:1050F000C4F82851C4F80052681EC4F808030120FF
:10510000FBF773FA124FB868007D50B11148006880
:105110004042B075C4F81C510120A0610E498002C4
:1051200008600C4844380068F168884202D00B4897
:10513000FBF764FFB868C068002802D0BDE8F04102
:105140000047BDE8F0810000300900200010004059
:10515000200100204815004008F5014051040A00D4
:1051600010B52D4CD4F80C01012802D02B48FBF7C8
:1051700045FFD4F81001012803D02848401CFBF754
:105180003DFFD4F80001012803D02448801CFBF720
:1051900035FFD4F8040118B12048C01CFBF72EFFDE
:1051A0000020C4F80C01C4F81001C4F80001C4F8D0
:1051B0000401C4F808010221C4F800120121C4F856
:1051C00008130822C4F80423154A0323154C13704E
:1051D00010755060606890B1027912B1FFF7E0FE7F
:1051E0000DE002785AB1027B437B807B01FA02F228
:1051F00001FA03F381400C481A430A430260A06895
:10520000006900B18047A0688068002802D0BDE82E
:105210001040004710BD000000100040F3030A00DA
:10522000300900202001002008F501402DE9F0415F
:105230002A4DD5F80001012802D02948FBF7DEFEEF
:10524000D5F80401012803D02548401CFBF7D6FE01
:1052500024480168244801700021C5F80011C5F8F0
:105260000411C5F80811491EC5F808130126C5F830
:10527000046381681D4F097D09B1B102396044683A
:1052800014B3207900B3617BDFF86480A06808EB79
:10529000C10100F5A070C1F810056279E179607B69
:1052A00000F06CFB607B06FA00F03860207B11494F
:1052B00008EBC000C0F810156279E179207B00F09E
:1052C0004BFB207B86403E600B480649091FC068A7
:1052D00008600B20C5F80002BDE8F0810010004016
:1052E000BD030A00081500402001002004F501401C
:1052F00000F001400C1100403009002070B5012081
:10530000FBF77EF90120FBF770F9144C4FF0FF30EA
:10531000C4F808030026C4F80062C4F81061012034
:105320002061A0610E4D2878012813D0022813D0E7
:10533000032811D05FF00100FDF768FEC4F810618A
:105340002E706E75002000F0DFF9BDE8704001207E
:10535000FBF76CB90620EFE70220EDE700100040F4
:10536000300900200148007870470000200100202B
:1053700001F03F014FF4003343EA01218300094863
:105380001844C0F81015D0F810150AB941F480116E
:10539000C0F81015D0F8101541F00301C0F8101531
:1053A000704700000060004008480069012806D0EE
:1053B000022806D0032806D00548FBF71FBE00F0E0
:1053C00095B800F007B800F0F1B8000030090020EF
:1053D00033050A002DE9F047DFF8F08004210120B1
:1053E00088F80010D8F81810491CC8F81810FBF7F6
:1053F000FCF837480068374D2870374C0026C4F851
:105400000C61C4F80061C4F81061C4F80461A868B4
:10541000DFF8C8900127007DA0B130480838006847
:10542000400502D42E48FBF7E9FD294840300068CA
:10543000404288F81600C4F81C61A7614FF48061EF
:10544000C9F80010D4F8000118B125480930FBF75D
:10545000D5FDD4F80C0118B121480A30FBF7CEFD78
:105460004FF0E020B046D0F8000210F0020F03D059
:105470001B480B30FBF7C2FD6E68CEB13078B8B177
:10548000C4F80C81717B184A164802EBC101C1F8BF
:1054900010057278F178707B00F05EFA707B0F492E
:1054A00007FA00F0091F0860F07B8740C9F8007018
:1054B000A868C06800B18047A868417D002903D072
:1054C00003490068091F0860BDE8F0873009002023
:1054D00008150040200100200010004008F50140A0
:1054E000C0040A000C11004000F001402DE9F04119
:1054F000294C0026C4F80C61C4F80061C4F810619E
:10550000C4F80861C4F80461012004F58074FBF755
:105510006CF80820C4F804020125C4F808520720DA
:10552000C4F800011D484468002C32D0207920B115
:10553000207B1B4905FA00F008602078002828D05D
:10554000A068C0F84061A17B164FA06807EBC101BD
:1055500000F5A070C1F810056278E178A07B00F03A
:105560000DFAA068C0F84061E17B0F4807EBC1016C
:10557000C1F81005E17BA06807EBC101C1F8140573
:10558000A17B05FA01F0E17B8D4005492843091F05
:105590000860BDE8F08100000010004020010020FC
:1055A00008F5014000F001400C11004070B5234C9B
:1055B000D4F80C01012802D02148FBF71FFDD4F8D4
:1055C0001001012803D01E48401CFBF717FDD4F83A
:1055D0000001012803D01A48801CFBF70FFD0020B2
:1055E000C4F80C01C4F81001C4F80001C4F80401A7
:1055F000411EC4F80813C4F80002124C626872B16C
:10560000117861B1557B012303FA05F1957BD27BBB
:1056100003FA05F593400C4A2943194311600B49DD
:10562000032208704A7048600875A0680069002865
:1056300002D0BDE87040004770BD0000001000407F
:10564000F5040A002001002008F50140300900207F
:1056500070B506460C460120FAF7D2FFFFF74EFE62
:10566000244D25482649C5E9014600240470032637
:105670004670446004610475447584751F48086071
:105680001E48F030091F08601E48016821F0010122
:1056900041F0807101600120FAF7C8FF686838B3F3
:1056A000017909B9017819B38168C1F80865042244
:1056B000C1F81025027CC2F18102C1F8402540F2F8
:1056C0000112C1F80022C1F804450122CA60C1F8E4
:1056D0004041017921B142798179C079FFF748FED3
:1056E0006868017821B142788178C078FFF740FE80
:1056F000014870BD20010020300900201410004036
:1057000064F50140741700402DE9F041174C002565
:105710000746C4F80052164E307803281CD0681E85
:10572000C4F80803C4F80C51032070700120FAF784
:105730005CFF00BFC4F80051C4F81051C4F8045114
:1057400075603575002F0FD00A4880680069002801
:105750000AD0BDE8F04100476FF00800C4F8080324
:105760000820C4F80403E5E7BDE8F081001000401C
:1057700030090020200100202DE9F0470746DFF81E
:10578000908022484FF0FF3100EB0716C8F808134D
:105790000120FAF72AFF1F4C0025DFF87C90657581
:1057A0006770D9F80800032F0268A2604168C4E955
:1057B0000315A5613068606019D2337AC8F80032E9
:1057C000C8F80C51C8F81051F37A14481BB10160A5
:1057D000006828B108E00260006828B9104801E0BC
:1057E0000F48401DFBF70AFC717AC8F80413D9F87A
:1057F0000800007D28B1022F03D10A49A57578025F
:10580000086001206075BDE8F08700006873000043
:105810000010004030090020200100200415004045
:105820009C020A0004F501402DE9F05F404C8246DD
:105830004048667800EB0617607D012802D03E489C
:10584000FBF7DCFB207D18B13B48401CFBF7D6FB87
:10585000012500212575DFF8E490A0466175032E2F
:1058600047D2BAF1000F3CD1D9F80440BCB3227939
:10587000AAB38A460846A168C1F84001217BDFF837
:10588000C0B0A0680BEBC10100F5A070C1F8100515
:105890006279E179207B00F071F82A49C1F80CA106
:1058A000607B29490BEBC000C0F810156279E179E3
:1058B000607B00F051F8217B627B05FA01F005FA6C
:1058C00002F1084321490860D9F80400204A81798F
:1058D0001268CA4012F0010F01D180680560386873
:1058E0000560022E01D0012E07D1B97A88F8001088
:1058F00003E011482530FBF781FBD9F80800007D53
:10590000002813D0022E11D110480068400503D49E
:1059100009482A30FBF772FB0E480068002805D1C1
:10592000BDE8F05F04482B30FBF768BBBDE8F09F93
:105930003009002068730000B8020A00200100202E
:1059400000F00140001000400C11004004F501403F
:105950001005005004150040064B03EBC0000AB1CF
:10596000054A01E0044A303A02EB8101C0F81415FF
:105970007047000000F0014060600040064B03EB00
:10598000C0000AB1054A01E0044A303202EB81014D
:10599000C0F814157047000000F00140306000406E
:1059A0000348D0F80401012800D00020704700000F
:1059B0000010004030B5124B01460020D3F81044CF
:1059C000224609E0157A854205D1401C0A28F7DBFA
:1059D0004FF0FF3030BD5268002AF3D1421CF9D09D
:1059E0000872D3F810242AB152684A60D3F8102400
:1059F000516030BD0022C3F810144A6030BD000071
:105A000054040020F0B595B01C4615460F460846D4
:105A10001A9E00F009FB182109A8FAF79CFC0E96C3
:105A2000CDE909540023082203A9384600F011FBF0
:105A300005980690BDF81000ADF81C00BDF81200E6
:105A4000ADF81E0000208DF821000398082600F014
:105A50000300012802D0022818D032E00398334610
:105A6000850AC0F3C2008DF8200003980FA9C0F387
:105A70008314A200384600F0ECFA09A8009006ABA7
:105A800022460FA9284600F02BFA1AE00398840D4D
:105A9000C0F3C2008DF82000082C01D2254600E09A
:105AA000082533462A460FA9384600F0D2FA2E447C
:105AB000641B09AB06AA29460FA800F063F9002C65
:105AC000EAD1384600F0B6FA15B0F0BD70470120B3
:105AD00001F060BA084810B50178084A515C19B164
:105AE000001D00F091FF02E00C3000F09FFEBDE8C9
:105AF0001040002001F04EBA4400002000000020B9
:105B000008B5034A00924023024AFFF77BFF08BD15
:105B1000C16C0000540300200A4A012902EBC000B6
:105B200007D0022907D0032907D0042907D0002075
:105B30007047022070470420704700797047407911
:105B400070470000DC74000010B5FFF7C0FF0421AF
:105B50000348FFF72FFF02490120487210BD0000E3
:105B6000580000202DE9F0478CB0FBF701F918B17F
:105B700000200CB0BDE8F087784C0020C4F8180471
:105B8000BFF34F8F60680290A5684FF0000828406F
:105B900004EB800008E021680298814201D861602E
:105BA000E6E7284004EB80000C3002A9FCF75EFE1B
:105BB0000028F0D103AB029901EA050204EB82024E
:105BC000491CD26843F82020401C02910228F2D3DD
:105BD000039800F00300022802D001284ED0A5E06F
:105BE00003985022810D8946B2EB905F00D8502176
:105BF0000E4666F39F5003900831594800F0CBF9E8
:105C0000070078D000F010FA4346082203A938466E
:105C100000F025FA029908F1080A2940681A800064
:105C2000001D864223D94D4D0C3530B1C2B204EB74
:105C30008101301A90460C3104E02946F2B2002569
:105C400090462846C6B25346384600F008FA0AEB9A
:105C500008032DB1324629464FEA070000F0FFF94C
:105C6000029909F1030001EB900002903AE004EB85
:105C700081015346324638460C31EFE70398C0F3B2
:105C80008311062900D3062161F389100390C0F324
:105C90008310801C8100324800F07DF9070045D058
:105CA00000F0C2F94346082203A9384600F0D7F9AC
:105CB00008F1080800260FE00298434600EA0501B3
:105CC000401C04EB81010290042238460C3100F0A4
:105CD000C6F908F10408761C0398C0F38310B0429B
:105CE000EAD847B1D4F81054D4F8180468B138464B
:105CF00000F0A0F92CE019E0687A012804D12A68A4
:105D000028463946126890476D68002DF4D1384610
:105D100000F090F90020FAF7EEFED4F8180408B964
:105D2000029860600020FAF7E8FE11E0D4F8104411
:105D300004E021682046896888476468002CF8D10F
:105D400008480221008801EB004007A100F016F886
:105D5000FBF70EF880F001000BE700005404002070
:105D60000C750000580100204261636B656E64731E
:105D700020666C75736865640000000000231A4695
:105D800000F0BEBF2DE9F0470E4680461C46924605
:105D900008293ED894F80C9000202073194610462C
:105DA00000F0E8FE0025B54206D218F805201AA139
:105DB0002046FDF7D7FB03E019A12046FDF7D2FBF3
:105DC0006D1C082DEFD317A12046FDF7CBFB002556
:105DD000B54210D218F80570FAF7A0FA0068C05D55
:105DE00010F03E0F01D03A4600E02E220EA12046D0
:105DF000FDF7B8FB03E00DA12046FDF7B3FB6D1CDA
:105E0000082DE5D301222146504600F095FE84F886
:105E10000C90BDE8F08700002025303278000000AB
:105E2000202020007C0000002563000020000000EE
:105E3000104810B5FF218160002101604160C0F869
:105E40001814C0F8141480F820140B4800F0F0F86F
:105E500000280DD109480A490A4B401AC108002000
:105E600003E000BF23F82000401C8842FAD3002042
:105E700010BD0000540400200C7500000C750000DB
:105E8000DC7400004401002002480349401AC008A5
:105E9000704700000C750000DC74000013B5684604
:105EA000FCF7E6FE08B100201CBD0248009950F83E
:105EB00031001CBDDC74000070B508480125D0F825
:105EC000104480F8205405E0657221682046496836
:105ED00088476468002CF7D170BD0000540400208E
:105EE0002DE9FF4781460C9D00200C462F7B28732F
:105EF000984616462946184600F03CFE072E42D228
:105F0000DFE806F004090F161F2A36004946284626
:105F1000FDF728FB37E0494628462268FDF722FBBB
:105F200031E0D4E9002349462846FDF71BFB2AE06F
:105F3000A0680090D4E9002349462846FDF712FBEB
:105F400021E0D4E90201CDE90001D4E9002349466A
:105F50002846FDF707FB16E004F1080007C88DE8A6
:105F60000700D4E9002349462846FDF7FBFA0AE07A
:105F700004F108000FC88DE80F00D4E9002349465A
:105F80002846FDF7EFFA00222946404600F0D4FDEE
:105F90002F73BDE8FF872DE9F041858A80462D1FCC
:105FA0004819C01CB0FBF5F0C6B24046FCF764FFD0
:105FB000041E19D00020207101206071E5800027A7
:105FC0002546761EC4F800800BE04046FCF754FFDF
:105FD00060B16179491C6171286005467F1CC0F879
:105FE0000080B742F1D32046BDE8F081204600F0A2
:105FF00002F80020F8E72DE9F041457901466B1ED3
:10600000002201E00968521C9A42FBD30F68014646
:10601000002605E038460C68FCF74DFF2146761C4B
:10602000AE42F7D3BDE8F0810121001DFCF708BFA7
:10603000FCF756BF10B504460121001DFCF716FF02
:1060400010F0FF0F04D12046BDE81040FFF7D3BF8A
:1060500010BD38B501240094FCF7CEFD38BD38B52D
:1060600000240094FCF7C8FD38BD000070B51A4C40
:106070000546206810B91948FAF7C0FFD4F8D400D3
:106080000A2803D31548401CFAF7B8FFD4F8CC000F
:1060900000EB800004EB800115F8040B08712DCD96
:1060A0008860CA600B614D61D4F8D400401CC4F80C
:1060B000D400D4F8CC00401CC4F8CC00D4F8CC10E8
:1060C00000200A2901D3C4F8CC004FF0E0214FF49E
:1060D0000010C1F8000270BD4C0900204A000B00FE
:1060E00010B5040002D10948FAF788FF084941F8C1
:1060F000CC4B002041F874098867C8674FF0E02155
:106100004FF40010C1F8000110BD00003E000B006C
:106110004C09002010B5074CD4F8D4000A2802D945
:106120000548FAF76BFFD4F8D400C0F10A00C0B2FA
:1061300010BD00004C09002079000B000949022223
:106140000A60BFF36F8FBFF34F8F0A1D10600648C0
:106150000268002AFCD000200860BFF36F8FBFF3F5
:106160004F8F704704E5014000E4014010B500F096
:1061700003029043D200FF24944003689140A3435C
:10618000CA18094901230B60BFF36F8FBFF34F8F0C
:10619000026006480268002AFCD000200860BFF3B5
:1061A0006F8FBFF34F8F10BD04E5014000E4014045
:1061B000F0B515460E460746002404E0315D381957
:1061C000FFF7D4FF641CAC42F8D3F0BD0148C068AF
:1061D00070470000240A00200148806870470000D2
:1061E000240A00200148406870470000240A00206B
:1061F000014981F881007047240A0020FCF7DCBFC8
:1062000070B5FCF7DFFF00240E4E2546204600F057
:1062100053FC04F1080000F04FFC3555641C082CB9
:10622000F4D309480121057045608560C5600561AA
:10623000456180F8805080F85850C56780F881101B
:1062400070BD00002C010020240A0020FCF7E6BFEE
:10625000FDF78AB82DE9FF4F81B0444FDDE90EA864
:1062600003260025F86F0C46AB4610B94048FAF7F4
:10627000C5FE3878032803D03D48401CFAF7BEFE1F
:10628000F86FB9464178C8072FD199F8810060B3FB
:1062900000270198E8B3039A584662F31700C1F348
:1062A000410161F31F6009EB84018A6BCAF800B0F9
:1062B000C8F800B00090904234D0204600F024FC92
:1062C000051E07EA05072DD004F1080109EB81023C
:1062D0000099916104990D4223D0264E305D00B3A0
:1062E000204600F032F910B105E00127D1E720483F
:1062F0002830FAF783FE204600F029F9CAF800009A
:10630000BAF1000F0AD018B919482E30FAF776FE04
:1063100000E01BE006F804B0022603E01448323027
:10632000F4E7012677B1204600F02DF9C8F8000007
:1063300018B110480121015506E00C485830C8F842
:10634000000001E0C8F800B00DB107E004264C469B
:10635000D9F87C00FCF762FFC4F87CB089F800B083
:1063600000F068F805B03046BDE8F08F240A002040
:106370002D010C002C01002010B50C4C207810B120
:106380000B48FAF73BFE00F0B3FB00280DD0FF22CC
:106390000270417841F00601417000214318491C08
:1063A0009A702029FAD30321217010BD240A0020FD
:1063B00007010C0070B51A4C05460E4620780128DE
:1063C00004D0022802D01748FAF718FEB5B1207899
:1063D000012803D01348401DFAF710FEE06818B9F1
:1063E0001048801DFAF70AFEE068007820B1606866
:1063F00000F08AFB022502E0002500E004254EB1F2
:10640000606800F0A4F8A168814203D005481D30FF
:10641000FAF7F4FD0020207000F00CF8284670BD5B
:10642000240A0020CC000C00014890F8800070473E
:10643000240A00202DE9F041104C207800281AD1C0
:1064400094F88000002816D10825012600276069ED
:10645000FCF70EFF18B184F8806060692061606904
:10646000401C6061082800D1676194F88000002812
:1064700001D16D1EEBD1BDE8F0810000240A00209F
:1064800070B5224C207810B12148FAF7B7FD94F886
:1064900080000025F8B12069606000F074F8A06009
:1064A00018B91B48C01DFAF7A9FDA0684078C007BD
:1064B00005D194F8810010B10220E56009E0606820
:1064C00000F02BF8032806D200F012FBE06010B1B8
:1064D0000120207002E02078002815D0A06818B9AB
:1064E0000B482030FAF78AFD2069606004EB8000D9
:1064F000C17E491CC17684F88050C27EA068417874
:1065000062F342014170012070BD0000240A0020A6
:1065100098000C000830FCF72FBE0830FCF7A8BE2E
:106520000830FCF7B5BE0830FCF702BF0148007820
:1065300070470000240A002010B5044600F0C4FA99
:106540002046BDE81040FCF717BEFCF791BE70B5C1
:106550000446FCF79DFE050002D0204600F0B4FA88
:10656000284670BD70B50E4604460025FCF724FE93
:1065700038B121463046FCF7ADFE10B1FFF75AFFA7
:106580000125284670BDFCF7D3BE00000148007805
:106590007047000034010020044801788170417880
:1065A0000170001D50F82100004700003401002058
:1065B000024988704870087070470000340100205C
:1065C00001484078704700003401002010B50446AF
:1065D000022802D30248FAF711FD0248447010BDA8
:1065E00033000D00340100204058002800D0012065
:1065F000704708B5002242504058009008BDD0F8BE
:106600000403084000D0012070474058002800D003
:106610000120704708B5002242504058009008BD44
:10662000002802D00149800108477047017300002B
:106630000121B1EB507F01D101207047002070474C
:1066400070B50D4600F0E2FA04000FD00020FAF712
:1066500052FA207920B10020FAF74FFA112070BDCC
:106660000120256020710020FAF747FA002070BD54
:1066700010B500F0CBFA002802D0002101600171B2
:1066800010BD00000149024800F0ACBCF801002038
:10669000002000402DE9F0410546007916460F46DE
:1066A00000EB40012D4A01EBC00102EB810494F89C
:1066B0002A1011B10820BDE8F081294951F82010B5
:1066C0002868FFF7BDFF08B11120F4E739462846D6
:1066D000FAF728FA66603869206030004FF001064A
:1066E0002FD03F7F4FF48E712868FFF782FF4FF461
:1066F000A2712868FFF77DFF28681A49C0F80413C3
:1067000028684FEA4711000B40B2002806DA00F073
:106710000F0000F1E02080F8141D03E000F1E020FC
:1067200080F800142868000B40B200F01F0206FA3F
:1067300002F14009800000F1E020C0F88012C0F8AA
:10674000001128680421C0F800150020A061E06154
:1067500084F8290044F8140FA675ACE7F80100206E
:10676000F4720000800002002DE9F0470546007930
:106770000B4600EB400101EBC000234901EB800414
:10678000284600F043F810B11120BDE8F0874FF023
:106790000008C4F82080A360626184F828804FF468
:1067A0008E76474631462868FFF723FF28684FF06A
:1067B0000109C0F808902146286800F0AFFB606826
:1067C00000BBD5F800A00EE094F8280008B10F2710
:1067D00016E031465046FFF707FF0028F4D0214667
:1067E000504600F09BFB216A60698142F1D331463B
:1067F0002868FFF7F9FE0028F9D02868C0F80C9047
:10680000C4F814803846C0E7F8010020007900EB96
:10681000400101EBC000044901EB80004069002801
:1068200000D0012070470000F80100202DE9F0475A
:10683000044600794FF0000900EB400101EBC00075
:10684000254901EB80072068C0F80095786880B181
:1068500020682249C0F8081320680121000B40B2CB
:1068600000F01F0291404009800000F1E020C0F8D4
:1068700080112068D0F80C25D0F81485D0F8086570
:10688000D0F810554FF0FF31C0F81415C0F80C15B2
:106890002068C0F80815C0F81015501C02D010462A
:1068A000FCF7B1FFB8F1FF3F02D04046FCF7ABFF69
:1068B000681C02D02846FCF7A6FF701C02D03046A8
:1068C000FCF7A1FF2068FFF7D3FE87F82A90C7F8EE
:1068D0000490BDE8F0870000F80100208402020067
:1068E0000149024800F02ABC240200200020004098
:1068F0002DE9F0410546164600790F46154A00EB92
:10690000C00102EB810494F8201011B10820BDE809
:10691000F081114951F820102868FFF791FE08B165
:106920001120F4E739462846FAF737F966603869E6
:1069300020601EB1397F2846FBF758FF28680821E0
:10694000C0F800150020A061E0610121606184F8B9
:106950002010DCE724020020F87200002DE9F04747
:1069600004460E460079204900EBC00001EB80058B
:1069700017463046FFF75CFE30B1204600F036F88F
:1069800020B11120BDE8F0871020FBE76F61AE60F9
:106990004FF49076002731462068FFF73BFE4FF416
:1069A000AC7841462068FFF735FE2068AA6869691F
:1069B000C0F84425C0F84815206801218160686846
:1069C00078B9B14649462068FFF71FFE06464146A2
:1069D0002068FFF71AFE0643F4D000B10F2700200D
:1069E00068613846CEE7000024020020007905499E
:1069F00000EBC00001EB80004069002800D00120BE
:106A000070470000240200202DE9F0470446007979
:106A1000274900EBC00001EB800720684FF0000918
:106A2000C0F80095786880B120682249C0F8081342
:106A300020680121000B40B200F01F029140400984
:106A4000800000F1E020C0F880112068D0F80C250B
:106A5000D0F81485D0F80865D0F810554FF0FF3104
:106A6000C0F80C15C0F814152068C0F80815C0F857
:106A70001015501C02D01046FCF7CEFEB8F1FF3FB7
:106A800002D04046FCF7C8FE681C02D02846FCF73E
:106A9000C3FE701C02D03046FCF7BEFE2068FFF734
:106AA000E7FD87F82090C7F80490BDE8F087000064
:106AB0002402002010030200024A002102EB8000A1
:106AC00081617047240A002010B50446064890F8FA
:106AD000801021B10069A04201D1FFF7ABFC03494E
:106AE0000020085510BD0000240A00202C010020C1
:106AF00010B5044CE06F002802D1FCF735FCE067CC
:106B000010BD0000240A002070B5094D0446E86F4E
:106B100010B90848FAF772FA04F10801E86FFCF7B7
:106B2000D9FB002802D00020E867012070BD0000DA
:106B3000240A00202E020C0010B50C46017A05290B
:106B400008D0407A38B1084808A102682046FCF70E
:106B500009FD00E01AB106A12046FCF703FD20461E
:106B6000BDE81040FCF70BBD90000020257300002D
:106B70000D0A000038B5C3880D46044633B114A091
:106B8000009015A216A12846FCF7ECFC217A0529F5
:106B90001CD0607A48B1A088FEF7BEFF164951F8B4
:106BA000202016A12846FCF7DDFCA0880021FFF775
:106BB00075F903461049207A143951F8202001B0A4
:106BC0002846BDE830400EA1FCF7CCBC38BD000023
:106BD0001B5B306D000000001B5B313B33316D00EF
:106BE00025734C6F67732064726F70706564202822
:106BF00025642925730D0A009000002025730000EC
:106C00003C25733E2025733A20000000034988424A
:106C100001D1034870470020704700000020004069
:106C20002000002070B5012670044FF0E0210025FF
:106C3000C1F88001084C4010C4F84803C4F80803A8
:106C400066602F20FFF7ECFCA660044C2F20A560A7
:106C5000FFF7E6FCA57070BD001001402800002081
:106C600070B5054688690C4600284FF484712846A3
:106C70000AD0FFF7BEFCD5F81805626AE1688854AF
:106C8000606A401C606270BDFFF7B3FCD5F8180560
:106C900070BD1FB501238DF80030CDE90121D0E989
:106CA0000012684690471FBD1FB501238DF80030C4
:106CB0008DF808100192D0E90012684690471FBD78
:106CC00070B50D4C0020D2B22070201D0B4D037802
:106CD000EB5C1BB1001DFFF741FE02E00C30FFF73B
:106CE00043FD08B1F9F7FCFE6078002802D0217856
:106CF0000029FAD070BD00004000002000000020F4
:106D00002DE9F84F204D92468946064698460122C5
:106D100069461846AF68F9F7D7FF58B300980021C5
:106D20000446801C09E000BF00EA07035AF821204E
:106D300005EB8303401C491CDA604145F4D34FEA5C
:106D4000164AFAF77DF84AEA0041601C384005EB24
:106D500080003C4005EB8402C160D06866F3C5004A
:106D600068F3891069F39F2020F00300401C20F095
:106D70000400D06095F8200402E000BFFEF7F2FEA8
:106D80000028FBD1BDE8F88F540400202DE9F84F0E
:106D90001D4C00256846D4E901A6FAF75BF80027E8
:106DA00038B30023009A61681CE0D1F800C008469F
:106DB000944503D9ACEB02020A6015E0A2EB0C0289
:106DC00063440760D0F80CC0C1698146BCF1000F74
:106DD00008D006EB030828F07F48C0E9018CC9F809
:106DE0001C5005460029E0D128466160FBF764FD90
:106DF00003E02846FBF760FD10B15046F9F7CAFFE3
:106E0000E770BDE8F88F0000280000200D4B10B59A
:106E1000596831B102680C68A24204D8A21A0A600B
:106E2000C161586010BD0B4603E00B46C969121BD7
:106E300021B10C689442F8D3A41A0C600260C161BD
:106E4000D86110BD280000202DE9F041144E77686C
:106E50003D462C4603E0844204D02546E469002CDC
:106E6000F9D11BE0D4B1A5420BD1F869706040B9EB
:106E70000C49012088600021B160F0702F20FFF7DD
:106E8000CFFB2168E069E86110B10268114401603C
:106E90007068874202D00120BDE8F0810020FBE746
:106EA00028000020001001402DE9F041194D6C68C8
:106EB000002C2CD0184800270068A968B846401A52
:106EC00020F07F462068B0420CD82146361A07448D
:106ED000E469087C20B181F8108088694969884795
:106EE000002CEFD129786878814206D1401CC0B2CD
:106EF0006870022801D185F80180064869780C3055
:106F000040F82170BDE8F0411420F9F79ABBBDE8C4
:106F1000F0810000280000200415014070B50C46E7
:106F200005464FF48E71FFF764FB216AA068415C4F
:106F3000206A401C2062C5F81C1570BD1FB50022D8
:106F40008DF800200291816801914261D0E9001220
:106F5000684690471FBD00001FB50A4601788DF8AE
:106F6000001041680191017A8DF80810C068039003
:106F7000044850F82210083850F8222068469047FC
:106F80001FBD00000C00002001490120087070475F
:106F90004000002010B588B0044620220E49684603
:106FA000F9F7C0F906200090C01F019002900390ED
:106FB0004FF0EB7006900CB1084A00E000226946E1
:106FC0000748FCF761F808B1F9F78AFD0448001F8B
:106FD000447008B010BD000024730000896F0000E9
:106FE000440000202DE9FF470C4605464FF4007190
:106FF000FFF705FB01274FF40178002618B34FF483
:10700000927949462846FFF7EFFAE0B1494628460B
:10701000FFF7EFFAC5F8088394F8290000B96F600C
:1070200002208DF80000D5F88004C5F88004039094
:10703000A0690290E0680190A661E661D4E90012BF
:107040006846904728E004212846FFF7D8FA18B38D
:107050004FF484712846FFF7C7FAE8B12146284665
:10706000FFF7FEFD616AA069884215D1E06938B179
:10707000E268616AA0612069E6616662E06008E03A
:1070800094F8290000B96F60C5F80883A661E2682A
:10709000616A2046FFF7FDFD4FF48E784146284691
:1070A000FFF7A2FA78B1206A6169884202D294F8A7
:1070B000280020B341462846FFF79BFA616911B1C9
:1070C0002046FFF73BFF4FF4A27841462846FFF7E2
:1070D0008BFA002818D041462846FFF78AFA94F820
:1070E000290000B12F60A06900280DD0A661E268D8
:1070F000616A04B02046BDE8F047FFF7CABD2146EB
:107100002846FFF70BFFDEE7BDE8FF871FB50A46FD
:1071100001788DF8001041680191017A8DF808100E
:10712000C0680390044850F82210083850F8222014
:10713000684690471FBD00000C0000202DE9FF416C
:107140000C464FF4927705463946FFF75EFA002663
:10715000C0B139462846FFF75DFA02208DF80000DD
:10716000D5F88004C5F880040390D5F83C058DF867
:107170000800E0680190A661E661D4E90012684663
:10718000904723E04FF4887739462846FFF73DFAC9
:10719000E0B139462846FFF73DFAD5F83C15A0691D
:1071A000884213D1E06960B1E268D5F8000220F0AE
:1071B0002000C5F80002E069A0612069E661E06096
:1071C00001E0A661E2682046FFF76EFD4FF4A2776A
:1071D00039462846FFF719FA60B139462846FFF7C5
:1071E00019FAA06930B1A661D5F83C152046E268CD
:1071F000FFF75AFD4FF4907739462846FFF705FA16
:10720000002813D039462846FFF704FA60690028A1
:107210000CD0D5F84C058DF800608DF80800A068FA
:1072200001906661D4E9001268469047BDE8FF818D
:107230002DE9F05F8346DDE90A4A994690460D46FE
:107240000846012703E000BFB0FBF8F07F1C404573
:10725000FAD2B94500D94F465FEACA7012D18CB153
:107260005FEA8A7002D5B9F1000F01D0202607E04D
:10727000302605E031465846641EF9F769FD0CB129
:10728000A742F7D35FF00106B9F1010F02D9A9F1C6
:10729000010903E0B5FBF6F0404502D306FB08F612
:1072A000F2E7DFF83C9000BFB5FBF6F000FB1655A7
:1072B00019F800105846F9F74BFDB6FBF8F6002E0A
:1072C000F2D15FEACA7009D0002C07D0A74205D2DC
:1072D00020215846641EF9F73BFDF5E7BDE8F09F15
:1072E000067300000D0E0F100B0C18190000005053
:1072F0000003005085660000E16800000000000007
:107300000338FDD8704730313233343536373839A9
:107310004142434445460000015B0000D55A00004D
:10732000CD5A0000FFFFFFFFFFFFFFFFFFFFFFFF42
:10733000FFFFFFFF00000000000000000000D6017A
:107340000701000032536601172D391A440C400D15
:10735000490D3E1A2D0C4D000000000000000000F9
:107360000338FDD8704700000010004010110040A5
:1073700003100000010000000010004000000000A9
:107380000B02040000000000041000400000000098
:107390000701030100000000004040404040404021
:1073A00040404141414141404040404040404040D8
:1073B000404040404040404040050202020202027C
:1073C00002020202020202020220202020202020CB
:1073D00020202002020202020202909090909090DF
:1073E000101010101010101010101010101010109D
:1073F0001010101002020202020288888888888811
:1074000008080808080808080808080808080808FC
:1074100008080808020202024000000099730000F8
:107420007761726E696E670064656275670000005F
:107430001B5B313B33306D001B5B306D0000000087
:107440001B5B313B33316D001B5B313B33326D00D5
:107450001B5B313B33336D001B5B313B33346D00C1
:107460001B5B313B33356D001B5B313B33366D00AD
:107470001B5B313B33376D00696E666F00000000A7
:107480006572726F720000004750494F544500000A
:10749000505253005541525400000000554152547F
:1074A0004500000062616C6C6F632E6C6F675F6DEE
:1074B000656D706F6F6C0000617070002475000066
:1074C000000000205C010000B8030000707500009F
:1074D0005C010020242B0000540A00008874000086
:1074E0000000000090740000000000009474000090
:1074F000000000009C74000000000000A474000064
:1075000000000003B8740000000003036C000020BA
:10751000640000206C00002094030020540100202F
:1075200018000000014A6420004054200040032756
:107530001873338074332074337874332874333879
:107540007433307433407433487433507433587424
:1075500033607433687403207074041190D003C2D4
:1075600005064404192A3F4D33394B031FFD4A00D9
:0400000500000201F4
:00000001FF
